:1000000000308A00E9290000831A0A28A500030E9F
:10001000A6000F288312A500030EA600A6140A0846
:10002000AD008A018313A50E0408A7002008A800CC
:100030002108A9002208AA002308AB002408AC006C
:1000400083128B1E25280B193A28270884002808BC
:10005000A0002908A1002A08A2002B08A3002C0850
:10006000A4002D088A00260E83008312250EA618F0
:1000700083160900B61C4028361C4028B610792883
:10008000361D45283A0885003611B61C5328361807
:10009000532837080F3C0319532837081F3C03190E
:1000A0005328B70AB610B70A37081F3C031865284B
:1000B000B701B80A38083B3C03186528B801B90AEB
:1000C00039083B3C03186528B901B70803196C28A7
:1000D0003708103C031D79283615BA01B7080319F3
:1000E0003A1438081D3C0318BA1439081D3C03188B
:1000F0003A15AE08031D8528AF08031D8528B008F2
:10010000031D8528B1080319A228FF30B207031C7C
:10011000B307031CB407031CB507B208031DA228CC
:10012000B308031DA228B408031DA228B508031DA7
:10013000A2283108B5003008B4002F08B3002E08FB
:10014000B200B6140B118A11252883169B019C134B
:100150001C141A088312BF003F087F39031DBA28F8
:10016000B501B401B301B201B101B001AF01AE01FB
:1001700036103429BF1FBE283614BF283610BF13CF
:10018000C3013D30C2000930C100C0013F08C400B6
:10019000C601C701C801C901CA01CB01C408031DBA
:1001A000D728FF30A000A100A200A3002C292030F6
:1001B000C500C5080319242964000310CA0DCB0D1E
:1001C000A001A101A20143088039A300A008031DDA
:1001D000F228A108031DF228A208031DF228A30893
:1001E0000319F528CA0A0319CB0A0310C00DC10D63
:1001F000C20DC30DCC010039A0004B080139A3008A
:1002000020082304031D0A294A08440203190A2965
:10021000031812294408CA020030031C0130CB0223
:100220000130CC000310C60DC70DC80DC90DCC0898
:10023000031922290130C6070318C70A0319C80A7F
:100240000319C90AC503D9284608A0004708A10018
:100250004808A2004908A3002308B1002208B00002
:100260002108AF002008AE00003483169501073046
:1002700083128500F830831685008312B701B80118
:10028000B90181013108B5003008B4002F08B3006E
:100290002E08B2003611B610C0308B0400340F3077
:1002A000A0008101813084000008F0390738800007
:1002B00064000008F739A019F039200480001F13EA
:1002C00083161F109F101F119F1183121F1083167A
:1002D0000108C73908388100853083129000073043
:1002E0009900831605086400831219088C1183167F
:1002F000990183128B16831681138312A52031086E
:10030000BF00103083169B008312310883169A00B9
:100310001C1583120B08A0008B13831655309D000B
:10032000AA309D009C149C1893291C11831220084C
:100330008B043008BF00113083169B0083123008F5
:1003400083169A001C1583120B08A0008B138316CA
:1003500055309D00AA309D009C149C18AD291C119D
:10036000831220088B042F08BF00123083169B00D5
:1003700083122F0883169A001C1583120B08A00005
:100380008B13831655309D00AA309D009C149C1839
:10039000C7291C11831220088B042E08BF001330BC
:1003A00083169B0083122E0883169A001C15831255
:1003B0000B08A0008B13831655309D00AA309D00BA
:1003C0009C149C18E1291C11831220088B043521F0
:1003D000F62984011F3083051F1383161F109F10F9
:1003E0001F119F110730831299004F29640085194E
:1003F0008A2A0B138B138B1BFA29FB30831685007B
:10040000033095009B019C131C141A088312BE0034
:10041000BE1B0E2A80303E07BC00122A3E087F39E0
:10042000803CBC00BD103D103D11BB018519872AE1
:100430006400BB0A05080339033C031D2A2A3D104A
:10044000BD113C083B020318272A0515292A05116E
:100450000000862A0518352A8518352ABD19342A40
:10046000BD158030BC003D15472A3D18472A0518A8
:10047000402A3C08013C0318402A3D15BC03472A8A
:100480008518472A3C0F452A472A3D15BC0A3D14CA
:100490003D1D862ABD143D113C087F3C03186B2A84
:1004A00080303C02BF0083169B0183123F088316F5
:1004B0009A001C1583120B08A0008B13831655306D
:1004C0009D00AA309D009C149C18642A1C11831264
:1004D00020088B04862A3C08803C8038C0008316A4
:1004E0009B018312400883169A001C1583120B0887
:1004F000A0008B13831655309D00AA309D009C14DC
:100500009C18802A1C11831220088B04162ABD18FF
:08051000A5203521F629630046
:024200000000BC
:104240000000010008000400000000000000000061
:02400E00C831B7
:00000001FF
